:100000000C942A001895000018950000189500001F
:10001000189500001895000018950000189500002C
:10002000189500001895000018950000189500001C
:10003000189500000C94572518950000189500009D
:1000400018950000189500001895000018950000FC
:10005000189500008FE58DBFC0E2E4E94E2E88E0E0
:100060008EBFD8E0F7E05F2EEEEFF7E0A0E6B0E05D
:10007000A89584B7082E877F84BF88E1992781BD22
:1000800091BD88278D933197E9F783E389B980E0A3
:1000900080BD88E18AB96624579A7894D29ADA9812
:1000A0008C988D9A95988E9A96988F988A9A92980D
:1000B00080917A02806480937A02E0E0F0E0ADED16
:1000C000B2E09CE00E944626A19AA998A69AAE9A10
:1000D000D59AD69AD79AAAEEB2E0E4EFFCE40E9451
:1000E00074240E943B2482E2A9EFB2E08D9388271A
:1000F0008C930E94B4080E94BF080E941D090E94B0
:100100001D095A924A9280E0A42DB52D8C9381E06E
:100110000E94D1235A924A9280E0A42DB52D8C934F
:1001200081E00E94D1230E94B009249682E00E94BF
:10013000CD235A924A92A42DB52DE2E0FDE40E940F
:1001400074248CE00E94D1230E94610A22968CE0E4
:100150000E94CD2384E690E00E945F245A924A9246
:1001600080E0A42DB52D8C9381E00E94D1235A927A
:100170004A9281E0A42DB52D8C9381E00E94D12379
:100180000E94B009249682E00E94CD235A924A929E
:10019000EAEEF2E0A42DB52D0E9421268FE00E9408
:1001A000D1230E94610A22968FE00E94CD2384E62B
:1001B00090E00E945F245A924A9280E0A42DB52DCF
:1001C0008C9381E00E94D1235A924A9283E0A42D1D
:1001D000B52D8C9381E00E94D1230E94B009249612
:1001E00082E00E94CD235A924A92A42DB52DEEE0D2
:1001F000FDE40E9474248FE00E94D1230E94610AD2
:1002000022968FE00E94CD2384E690E00E945F2436
:100210005A924A9280E0A42DB52D8C9381E00E94E1
:10022000D1235A924A9284E0A42DB52D8C9381E07B
:100230000E94D1230E94B009249682E00E94CD231F
:100240005A924A92A42DB52DEEE1FDE40E94742449
:100250008EE00E94D1230E94610A22968EE00E94C5
:10026000CD235A924A9280E0A42DB52D8C9381E043
:100270000E94D1235A924A9285E0A42DB52D8C93E9
:1002800081E00E94D1230E94B009249682E00E945E
:10029000CD235A924A92A42DB52DEEE0FDE40E94A2
:1002A00074248FE00E94D1230E94610A22968FE07D
:1002B0000E94CD23E5E0F0E00E942824DA9A959A86
:1002C0000E941D095A924A9280E0A42DB52D8C936C
:1002D00081E00E94D1235A924A9282E0A42DB52D4A
:1002E0008C9381E00E94D1230E94B009249682E081
:1002F0000E94CD235A924A92A42DB52DECE2FDE442
:100300000E9474248FE00E94D1230E94610A2296E9
:100310008FE00E94CD2380E0809377025A924A9228
:1003200080E0A42DB52D8C9381E00E94D1235A92B8
:100330004A9283E0A42DB52D8C9381E00E94D123B5
:100340000E94B009249682E00E94CD235A924A92DC
:10035000A42DB52DECE3FDE40E9474248FE00E94EF
:10036000D1230E94610A22968FE00E94CD238EE065
:1003700091E00E945F245A924A9280917702A42DC4
:10038000B52D8C9381E00E94D1235A924A9283E04A
:10039000A42DB52D8C9381E00E94D1230E94B00939
:1003A000249682E00E94CD235A924A92A42DB52D24
:1003B000ECE4FDE40E94742482E00E94D1230E94B8
:1003C000610A229682E00E94CD238EE091E00E9495
:1003D0005F245A924A9280917702A42DB52D8C9376
:1003E00081E00E94D1235A924A9283E0A42DB52D38
:1003F0008C9381E00E94D1230E94B009249682E070
:100400000E94CD235A924A92A42DB52DEEE4FDE42C
:100410000E94742482E00E94D1230E94610A2296E5
:1004200082E00E94CD238EE091E00E945F245A92E8
:100430004A9280917702A42DB52D8C9381E00E9481
:10044000D1235A924A9283E0A42DB52D8C9381E05A
:100450000E94D1230E94B009249682E00E94CD23FD
:100460005A924A92A42DB52DE0E5FDE40E94742431
:1004700082E00E94D1230E94610A229682E00E94BB
:10048000CD238EE091E00E945F245A924A9280919F
:100490007702A42DB52D8C9381E00E94D1235A922E
:1004A0004A9283E0A42DB52D8C9381E00E94D12344
:1004B0000E94B009249682E00E94CD235A924A926B
:1004C000A42DB52DE2E5FDE40E94742482E00E9493
:1004D000D1230E94610A229682E00E94CD238EE001
:1004E00091E00E945F24A7E7B2E08C918F5F8C932C
:1004F00000917702023011F00C94BB019598DA98C4
:100500005A924A9280E0A42DB52D8C9381E00E94EE
:10051000D1235A924A9282E0A42DB52D8C9381E08A
:100520000E94D1230E94B009249682E00E94CD232C
:100530005A924A92A42DB52DE4E5FDE40E9474245C
:100540008FE00E94D1230E94610A22968FE00E94D0
:10055000CD235A924A9280917702A42DB52D8C9387
:1005600081E00E94D1235A924A9283E0A42DB52DB6
:100570008C9381E00E94D1230E94B009249682E0EE
:100580000E94CD235A924A92A42DB52DE4E6FDE4B3
:100590000E94742482E00E94D1230E94610A229664
:1005A00082E00E94CD238EE091E00E945F245A9267
:1005B0004A9280917702A42DB52D8C9381E00E9400
:1005C000D1235A924A9283E0A42DB52D8C9381E0D9
:1005D0000E94D1230E94B009249682E00E94CD237C
:1005E0005A924A92A42DB52DECE4FDE40E947424A5
:1005F00082E00E94D1230E94610A229682E00E943A
:10060000CD238EE091E00E945F245A924A9280911D
:100610007702A42DB52D8C9381E00E94D1235A92AC
:100620004A9283E0A42DB52D8C9381E00E94D123C2
:100630000E94B009249682E00E94CD235A924A92E9
:10064000A42DB52DEEE4FDE40E94742482E00E9406
:10065000D1230E94610A229682E00E94CD238EE07F
:1006600091E00E945F245A924A9280917702A42DD1
:10067000B52D8C9381E00E94D1235A924A9283E057
:10068000A42DB52D8C9381E00E94D1230E94B00946
:10069000249682E00E94CD235A924A92A42DB52D31
:1006A000E0E5FDE40E94742482E00E94D1230E94D0
:1006B000610A229682E00E94CD238EE091E00E94A2
:1006C0005F245A924A9280917702A42DB52D8C9383
:1006D00081E00E94D1235A924A9283E0A42DB52D45
:1006E0008C9381E00E94D1230E94B009249682E07D
:1006F0000E94CD235A924A92A42DB52DE2E5FDE445
:100700000E94742482E00E94D1230E94610A2296F2
:1007100082E00E94CD238EE091E00E945F24A7E753
:10072000B2E08C918F5F8C9300917702063011F0CC
:100730000C94A9025A924A9280E0A42DB52D8C9374
:1007400081E00E94D1235A924A9282E0A42DB52DD5
:100750008C9381E00E94D1230E94B009249682E00C
:100760000E94CD235A924A92A42DB52DE6E6FDE4CF
:100770000E9474248FE00E94D1230E94610A229675
:100780008FE00E94CD23E6E7FDE40E941A240E9438
:1007900021245A924A9280917702A42DB52D8C93F0
:1007A00081E00E94D1235A924A9283E0A42DB52D74
:1007B0008C9381E00E94D1230E94B009249682E0AC
:1007C0000E94CD235A924A92A42DB52DE4E6FDE471
:1007D0000E94742482E00E94D1230E94610A229622
:1007E00082E00E94CD238EE091E00E945F24E6E744
:1007F000FDE40E941A240E9421240E94C7155A92E7
:100800004A9280917702A42DB52D8C9381E00E94AD
:10081000D1235A924A9283E0A42DB52D8C9381E086
:100820000E94D1230E94B009249682E00E94CD2329
:100830005A924A92A42DB52DECE4FDE40E94742452
:1008400082E00E94D1230E94610A229682E00E94E7
:10085000CD238EE091E00E945F245A924A928091CB
:100860007702A42DB52D8C9381E00E94D1235A925A
:100870004A9283E0A42DB52D8C9381E00E94D12370
:100880000E94B009249682E00E94CD235A924A9297
:10089000A42DB52DEEE4FDE40E94742482E00E94B4
:1008A000D1230E94610A229682E00E94CD238EE02D
:1008B00091E00E945F245A924A9280917702A42D7F
:1008C000B52D8C9381E00E94D1235A924A9283E005
:1008D000A42DB52D8C9381E00E94D1230E94B009F4
:1008E000249682E00E94CD235A924A92A42DB52DDF
:1008F000E0E5FDE40E94742482E00E94D1230E947E
:10090000610A229682E00E94CD238EE091E00E944F
:100910005F245A924A9280917702A42DB52D8C9330
:1009200081E00E94D1235A924A9283E0A42DB52DF2
:100930008C9381E00E94D1230E94B009249682E02A
:100940000E94CD235A924A92A42DB52DE2E5FDE4F2
:100950000E94742482E00E94D1230E94610A2296A0
:1009600082E00E94CD238EE091E00E945F24A7E701
:10097000B2E08C918F5F8C935A924A9280E0A42DC2
:10098000B52D8C9381E00E94D1235A924A9282E045
:10099000A42DB52D8C9381E00E94D1230E94B00933
:1009A000249682E00E94CD235A924A92A42DB52D1E
:1009B000EAE7FDE40E9474248FE00E94D1230E94A4
:1009C000610A22968FE00E94CD235A924A9280912A
:1009D0007702A42DB52D8C9381E00E94D1235A92E9
:1009E0004A9283E0A42DB52D8C9381E00E94D123FF
:1009F0000E94B009249682E00E94CD235A924A9226
:100A0000A42DB52DE4E6FDE40E94742482E00E944A
:100A1000D1230E94610A229682E00E94CD238EE0BB
:100A200091E00E945F245A924A9280917702A42D0D
:100A3000B52D8C9381E00E94D1235A924A9283E093
:100A4000A42DB52D8C9381E00E94D1230E94B00982
:100A5000249682E00E94CD235A924A92A42DB52D6D
:100A6000ECE4FDE40E94742482E00E94D1230E9401
:100A7000610A229682E00E94CD238EE091E00E94DE
:100A80005F24E6E7FDE40E941A240E94212488E204
:100A900090E00E945F24A2E3B2E0BA93AA930E947E
:100AA00089152296A2E3B2E0EAE8FDE40E946626F8
:100AB00011F00C9441050E94C7155A924A928091F8
:100AC0007702A42DB52D8C9381E00E94D1235A92F8
:100AD0004A9283E0A42DB52D8C9381E00E94D1230E
:100AE0000E94B009249682E00E94CD235A924A9235
:100AF000A42DB52DEEE4FDE40E94742482E00E9452
:100B0000D1230E94610A229682E00E94CD238EE0CA
:100B100091E00E945F245A924A9280917702A42D1C
:100B2000B52D8C9381E00E94D1235A924A9283E0A2
:100B3000A42DB52D8C9381E00E94D1230E94B00991
:100B4000249682E00E94CD235A924A92A42DB52D7C
:100B5000E0E5FDE40E94742482E00E94D1230E941B
:100B6000610A229682E00E94CD238EE091E00E94ED
:100B70005F245A924A9280917702A42DB52D8C93CE
:100B800081E00E94D1235A924A9283E0A42DB52D90
:100B90008C9381E00E94D1230E94B009249682E0C8
:100BA0000E94CD235A924A92A42DB52DE2E5FDE490
:100BB0000E94742482E00E94D1230E94610A22963E
:100BC00082E00E94CD238EE091E00E945F24A7E79F
:100BD000B2E08C918F5F8C935A924A9280E0A42D60
:100BE000B52D8C9381E00E94D1235A924A9282E0E3
:100BF000A42DB52D8C9381E00E94D1230E94B009D1
:100C0000249682E00E94CD235A924A92A42DB52DBB
:100C1000EEE8FDE40E9474248FE00E94D1230E943C
:100C2000610A22968FE00E94CD23EEE9FDE40E9446
:100C30001A2482E20E942424E8EAFDE40E941A2495
:100C400082E20E9424240E9421245A924A92809196
:100C50007702A42DB52D8C9381E00E94D1235A9266
:100C60004A9283E0A42DB52D8C9381E00E94D1237C
:100C70000E94B009249682E00E94CD235A924A92A3
:100C8000A42DB52DE4E6FDE40E94742482E00E94C8
:100C9000D1230E94610A229682E00E94CD238EE039
:100CA00091E00E945F245A924A9280917702A42D8B
:100CB000B52D8C9381E00E94D1235A924A9283E011
:100CC000A42DB52D8C9381E00E94D1230E94B00900
:100CD000249682E00E94CD235A924A92A42DB52DEB
:100CE000ECE4FDE40E94742482E00E94D1230E947F
:100CF000610A229682E00E94CD23E5E0F0E00E94A6
:100D000028240E94C7158EE091E00E945F245A9229
:100D10004A9280917702A42DB52D8C9381E00E9498
:100D2000D1235A924A9283E0A42DB52D8C9381E071
:100D30000E94D1230E94B009249682E00E94CD2314
:100D40005A924A92A42DB52DEEE4FDE40E9474243B
:100D500082E00E94D1230E94610A229682E00E94D2
:100D6000CD238EE091E00E945F245A924A928091B6
:100D70007702A42DB52D8C9381E00E94D1235A9245
:100D80004A9283E0A42DB52D8C9381E00E94D1235B
:100D90000E94B009249682E00E94CD235A924A9282
:100DA000A42DB52DE0E5FDE40E94742482E00E94AC
:100DB000D1230E94610A229682E00E94CD238EE018
:100DC00091E00E945F245A924A9280917702A42D6A
:100DD000B52D8C9381E00E94D1235A924A9283E0F0
:100DE000A42DB52D8C9381E00E94D1230E94B009DF
:100DF000249682E00E94CD235A924A92A42DB52DCA
:100E0000E2E5FDE40E94742482E00E94D1230E9466
:100E1000610A229682E00E94CD2384E690E00E943F
:100E20005F245A924A9280917702A42DB52D8C931B
:100E300081E00E94D1235A924A9283E0A42DB52DDD
:100E40008C9381E00E94D1230E94B009249682E015
:100E50000E94CD23A7E7B2E08C918F5F8C935A92CA
:100E60004A9280917702A42DB52D8C9381E00E9447
:100E7000D1235A924A9283E0A42DB52D8C9381E020
:100E80000E94D1230E94B009249682E00E94CD23C3
:100E90005A924A92A42DB52DE4E6FDE40E947424F2
:100EA00082E00E94D1230E94610A229682E00E9481
:100EB000CD2382E390E00E945F245A924A9280916F
:100EC0007702A42DB52D8C9381E00E94D1235A92F4
:100ED0004A9283E0A42DB52D8C9381E00E94D1230A
:100EE0000E94B009249682E00E94CD235A924A9231
:100EF000A42DB52DECE4FDE40E94742482E00E9450
:100F0000D1230E94610A229682E00E94CD2382E3CF
:100F100090E00E945F245A924A9280917702A42D19
:100F2000B52D8C9381E00E94D1235A924A9283E09E
:100F3000A42DB52D8C9381E00E94D1230E94B0098D
:100F4000249682E00E94CD235A924A92A42DB52D78
:100F5000EEE4FDE40E94742482E00E94D1230E940A
:100F6000610A229682E00E94CD2382E390E00E94F3
:100F70005F245A924A9280917702A42DB52D8C93CA
:100F800081E00E94D1235A924A9283E0A42DB52D8C
:100F90008C9381E00E94D1230E94B009249682E0C4
:100FA0000E94CD235A924A92A42DB52DE0E5FDE48E
:100FB0000E94742482E00E94D1230E94610A22963A
:100FC00082E00E94CD2382E390E00E945F245A9247
:100FD0004A9280917702A42DB52D8C9381E00E94D6
:100FE000D1235A924A9283E0A42DB52D8C9381E0AF
:100FF0000E94D1230E94B009249682E00E94CD2352
:101000005A924A92A42DB52DE2E5FDE40E94742483
:1010100082E00E94D1230E94610A229682E00E940F
:10102000CD2382E390E00E945F245A924A928091FD
:101030007702A42DB52D8C9381E00E94D1235A9282
:101040004A9283E0A42DB52D8C9381E00E94D12398
:101050000E94B009249682E00E94CD235A924A92BF
:10106000A42DB52DE0EBFDE40E94742482E00E94E3
:10107000D1230E94610A229682E00E94CD2382E35E
:1010800090E00E945F24A7E7B2E08C918F5F8C9381
:10109000009177020E3011F00C942F0780E08093BE
:1010A00077020E941D095A924A9280E0A42DB52D24
:1010B0008C9381E00E94D1235A924A9282E0A42D1F
:1010C000B52D8C9381E00E94D1230E94B009249613
:1010D00082E00E94CD235A924A92A42DB52DE2EBD4
:1010E000FDE40E9474248FE00E94D1230E94610AD3
:1010F00022968FE00E94CD230E94C715DA9AE2EC77
:10110000FDE40E941A240E94212482E390E00E94C0
:101110005F24ECECFDE40E941A240E942124E3E009
:10112000F0E00E942824DA980E94C7150E941D0949
:10113000DA9A0E94F11F0E94D7150E94A1220E94F4
:1011400045170E947B1B0E94FB1B0E94BA1D0E9438
:10115000D4190E945321DA98EAE0F0E00E94282492
:101160000C949808F894FFCFDF98EF93FF93E4EE88
:10117000F3E00E942E24FF91EF91DF9A0895DE980C
:10118000DD985A924A9281E2A42DB52D8C9381E08C
:101190000E94D1230E949E09229681E00E94CD23C5
:1011A0005A924A9288ECA42DB52D8C9381E00E942E
:1011B000D1230E949E09229681E00E94CD235A925B
:1011C0004A9286E0A42DB52D8C9381E00E94D12314
:1011D0000E949E09229681E00E94CD235A924A9253
:1011E00083E1A42DB52D8C9381E00E94D1230E9430
:1011F0009E09229681E00E94CD235A924A9280E273
:10120000A42DB52D8C9381E00E94D1230E949E09CC
:10121000229681E00E94CD235A924A928CE0A42D1E
:10122000B52D8C9381E00E94D1230E949E092296C5
:1012300081E00E94CD23DE9A089582E00E946E2410
:10124000DE98DD985A924A9280E2A42DB52D8C93B7
:1012500081E00E94D1230E949E09229681E00E9493
:10126000CD235A924A9280E8A42DB52D8C9381E02B
:101270000E94D1230E949E09229681E00E94CD23E4
:101280005A924A9280E4A42DB52D8C9381E00E945D
:10129000D1230E949E09229681E00E94CD23DD9AEF
:1012A00080E090E0A881B9818D939C93A881B98159
:1012B0000D911C91073F51E0150718F011F00C94A7
:1012C00077095A924A9280E0A42DB52D8C9381E043
:1012D0000E94D1230E94A709229681E00E94CD237B
:1012E000A881B9810E94D52310F40C945609DE9A86
:1012F00082E0481A8827580A229608955A924A92FC
:101300008DE0A42DB52D8C9381E00E94D1230E9405
:101310009E09229681E00E94CD2308955A924A9216
:101320008CE0A42DB52D8C9381E00E94D1230E94E6
:101330009E09229681E00E94CD230895DE98DD98D3
:1013400091E0A881B9810E943124DE9A0895DE9847
:10135000DD9A91E0A881B9810E943124DE9A089536
:1013600081E00E946E245A924A9280E2A42DB52D0B
:101370008C9381E00E94D1230E949E09229681E0F5
:101380000E94CD23EF93FF93E4EEF3E00E942E241E
:10139000FF91EF91DE98DD98AC81BD810C9146E024
:1013A000049FA881B9810C92A881B9818C91805841
:1013B0008C9391E0A881B9810E943124AA81BB81DC
:1013C0000C9140E4040FA881B9810C9391E0A881AD
:1013D000B9810E943124DE9A81E0481A8827580A90
:1013E0002296089582E00E946E2481E00E946E247D
:1013F000DE98DD985A924A9280E2A42DB52D8C9306
:1014000081E00E94D1230E949E09229681E00E94E1
:10141000CD235A924A9280E8A42DB52D8C9381E079
:101420000E94D1230E949E09229681E00E94CD2332
:101430005A924A9280E4A42DB52D8C9381E00E94AB
:10144000D1230E949E09229681E00E94CD23DD9A3D
:1014500080E090E0AA81BB818D939C93AA81BB819F
:101460000D911C91073F51E0150718F011F00C94F5
:101470005A0A0E94CA23A881B9810E947A240C9238
:101480000E94C7235A924A92AA81BB818C91A42DB3
:10149000B52D8C9381E00E94D1230E94A70922964A
:1014A00081E00E94CD23AA81BB810E94D52310F444
:1014B0000C942E0ADE9A83E0481A8827580A24964C
:1014C000089581E00E946E2482E00E946E2481E0F3
:1014D0000E946E2481E00E946E2481E00E946E24AE
:1014E000AA85BB850E946026A885B9858C9381E07A
:1014F000AC81BD818C93A885B9854C91AC81BD81AF
:101500000C91041718F011F00C94E212AC81BD811B
:101510008C91EA85FB8501E00A93AF81B8850E9432
:101520002626AE81BF81E6EDFDE40E94662611F01D
:101530000C94A00AE2EFF6E20E94C7230C949712E3
:10154000E8EDFDE40E94662611F00C94AD0AE8EF88
:10155000F6E20E94C7230C949712EAEDFDE40E9484
:10156000662611F00C94BA0AEEEFF6E20E94C72349
:101570000C949712ECEDFDE40E94662611F00C9499
:10158000C70AE4E0F7E20E94C7230C949712EEED3D
:10159000FDE40E94662611F00C94D40AEAE0F7E21A
:1015A0000E94C7230C949712E0EEFDE40E94662689
:1015B00011F00C94E10AE0E1F7E20E94C7230C94D9
:1015C0009712E2EEFDE40E94662611F00C94EE0AFA
:1015D000E6E1F7E20E94C7230C949712E4EEFDE4E3
:1015E0000E94662611F00C94FB0AECE1F7E20E94DF
:1015F000C7230C949712E6EEFDE40E94662611F0D4
:101600000C94080BE2E2F7E20E94C7230C949712B5
:10161000E8EEFDE40E94662611F00C94150BE8E25A
:10162000F7E20E94C7230C949712EAEEFDE40E94B1
:10163000662611F00C94220BEEE2F7E20E94C7231B
:101640000C949712ECEEFDE40E94662611F00C94C7
:101650002F0BE4E3F7E20E94C7230C949712EEEEFF
:10166000FDE40E94662611F00C943C0BEAE3F7E2DD
:101670000E94C7230C949712E0EFFDE40E946626B7
:1016800011F00C94490BE0E4F7E20E94C7230C949C
:101690009712E2EFFDE40E94662611F00C94560BBF
:1016A000E6E4F7E20E94C7230C949712E4EFFDE40E
:1016B0000E94662611F00C94630BECE4F7E20E94A2
:1016C000C7230C949712E6EFFDE40E94662611F002
:1016D0000C94700BE2E5F7E20E94C7230C9497127A
:1016E000E8EFFDE40E94662611F00C947D0BE8E51E
:1016F000F7E20E94C7230C949712EAEFFDE40E94E0
:10170000662611F00C948A0BEEE5F7E20E94C723DF
:101710000C949712ECEFFDE40E94662611F00C94F5
:10172000970BE4E6F7E20E94C7230C949712EEEFC2
:10173000FDE40E94662611F00C94A40BEAE6F7E2A1
:101740000E94C7230C949712E0E0FEE40E946626F4
:1017500011F00C94B10BE0E7F7E20E94C7230C9460
:101760009712E2E0FEE40E94662611F00C94BE0B94
:10177000E6E7F7E20E94C7230C949712E4E0FEE448
:101780000E94662611F00C94CB0BECE7F7E20E9466
:10179000C7230C949712E6E0FEE40E94662611F03F
:1017A0000C94D80BE2E8F7E20E94C7230C9497123E
:1017B000E8E0FEE40E94662611F00C94E50BE8E8F0
:1017C000F7E20E94C7230C949712EAE0FEE40E941D
:1017D000662611F00C94F20BEEE8F7E20E94C723A4
:1017E0000C949712ECE0FEE40E94662611F00C9433
:1017F000FF0BE4E9F7E20E94C7230C949712EEE096
:10180000FEE40E94662611F00C940C0CEAE9F7E263
:101810000E94C7230C949712E0E1FEE40E94662622
:1018200011F00C94190CE0EAF7E20E94C7230C9423
:101830009712E2E1FEE40E94662611F00C94260C59
:10184000E6EAF7E20E94C7230C949712E4E1FEE473
:101850000E94662611F00C94330CECEAF7E20E9429
:10186000C7230C949712E6E1FEE40E94662611F06D
:101870000C94400CE2EBF7E20E94C7230C94971201
:10188000E8E1FEE40E94662611F00C944D0CE8EBB2
:10189000F7E20E94C7230C949712EAE1FEE40E944B
:1018A000662611F00C945A0CEEEBF7E20E94C72367
:1018B0000C949712ECE1FEE40E94662611F00C9461
:1018C000670CE4ECF7E20E94C7230C949712EEE158
:1018D000FEE40E94662611F00C94740CEAECF7E228
:1018E0000E94C7230C949712E0E2FEE40E94662651
:1018F00011F00C94810CE0EDF7E20E94C7230C94E8
:101900009712E2E2FEE40E94662611F00C948E0C1F
:10191000E6EDF7E20E94C7230C949712E4E2FEE49E
:101920000E94662611F00C949B0CECEDF7E20E94ED
:10193000C7230C949712E6E2FEE40E94662611F09B
:101940000C94A80CE2EEF7E20E94C7230C949712C5
:10195000E8E2FEE40E94662611F00C94B50CE8EE75
:10196000F7E20E94C7230C949712EAE2FEE40E9479
:10197000662611F00C94C20CEEEEF7E20E94C7232B
:101980000C949712ECE2FEE40E94662611F00C948F
:10199000CF0CE4EFF7E20E94C7230C949712EEE21B
:1019A000FEE40E94662611F00C94DC0CEAEFF7E2EC
:1019B0000E94C7230C949712E0E3FEE40E9466267F
:1019C00011F00C94E90CE0E0F8E20E94C7230C94BB
:1019D0009712E2E3FEE40E94662611F00C94F60CE6
:1019E000E6E0F8E20E94C7230C949712E4E3FEE4D9
:1019F0000E94662611F00C94030DECE0F8E20E94C0
:101A0000C7230C949712E6E3FEE40E94662611F0C9
:101A10000C94100DE2E1F8E20E94C7230C94971297
:101A2000E8E3FEE40E94662611F00C941D0DE8E147
:101A3000F8E20E94C7230C949712EAE3FEE40E94A6
:101A4000662611F00C942A0DEEE1F8E20E94C723FD
:101A50000C949712ECE3FEE40E94662611F00C94BD
:101A6000370DE4E2F8E20E94C7230C949712EEE3EC
:101A7000FEE40E94662611F00C94440DEAE2F8E2BE
:101A80000E94C7230C949712E0E4FEE40E946626AD
:101A900011F00C94510DE0E3F8E20E94C7230C947E
:101AA0009712E2E4FEE40E94662611F00C945E0DAB
:101AB000E6E3F8E20E94C7230C949712E4E4FEE404
:101AC0000E94662611F00C946B0DECE3F8E20E9484
:101AD000C7230C949712E6E4FEE40E94662611F0F8
:101AE0000C94780DE2E4F8E20E94C7230C9497125C
:101AF000E8E4FEE40E94662611F00C94850DE8E40B
:101B0000F8E20E94C7230C949712EAE4FEE40E94D4
:101B1000662611F00C94920DEEE4F8E20E94C723C1
:101B20000C949712ECE4FEE40E94662611F00C94EB
:101B30009F0DE4E5F8E20E94C7230C949712EEE4AF
:101B4000FEE40E94662611F00C94AC0DEAE5F8E282
:101B50000E94C7230C949712E0E5FEE40E946626DB
:101B600011F00C94B90DE0E6F8E20E94C7230C9442
:101B70009712E2E5FEE40E94662611F00C94C60D71
:101B8000EEE2F7E20E94C7230C949712E4E5FEE42C
:101B90000E94662611F00C94D30DEAECF7E20E9445
:101BA000C7230C949712E6E5FEE40E94662611F026
:101BB0000C94E00DE2EDF5E20E94C7230C9497121D
:101BC000E8E5FEE40E94662611F00C94ED0DE8EDC8
:101BD000F5E20E94C7230C949712EAE5FEE40E9406
:101BE000662611F00C94FA0DEEEDF5E20E94C72383
:101BF0000C949712ECE5FEE40E94662611F00C941A
:101C0000070EE4EEF5E20E94C7230C949712EEE56E
:101C1000FEE40E94662611F00C94140EEAEEF5E242
:101C20000E94C7230C949712E0E6FEE40E94662609
:101C300011F00C94210EE0EFF5E20E94C7230C9402
:101C40009712E2E6FEE40E94662611F00C942E0E36
:101C5000E6EFF5E20E94C7230C949712E4E6FEE457
:101C60000E94662611F00C943B0EECEFF5E20E9408
:101C7000C7230C949712E6E6FEE40E94662611F054
:101C80000C94480EE6E4F7E20E94C7230C949712E6
:101C9000E8E6FEE40E94662611F00C94550EE2EE92
:101CA000F7E20E94C7230C949712EAE6FEE40E9432
:101CB000662611F00C94620EE2E0F6E20E94C72361
:101CC0000C949712ECE6FEE40E94662611F00C9448
:101CD0006F0EE8E0F6E20E94C7230C949712EEE63E
:101CE000FEE40E94662611F00C947C0EEEE0F6E213
:101CF0000E94C7230C949712E0E7FEE40E94662638
:101D000011F00C94890EE4E1F6E20E94C7230C94D2
:101D10009712E2E7FEE40E94662611F00C94960EFC
:101D2000EAE1F6E20E94C7230C949712E4E7FEE48E
:101D30000E94662611F00C94A30EE0E2F6E20E94E7
:101D4000C7230C949712E6E7FEE40E94662611F082
:101D50000C94B00EE6E2F6E20E94C7230C949712B0
:101D6000E8E7FEE40E94662611F00C94BD0EECE25A
:101D7000F6E20E94C7230C949712E0EBFDE40E9468
:101D8000662611F00C94CA0EE2E3F6E20E94C72325
:101D90000C949712EAE7FEE40E94662611F00C9478
:101DA000D70EE8E3F6E20E94C7230C949712ECE703
:101DB000FEE40E94662611F00C94E40EEAE6F7E2D7
:101DC0000E94C7230C949712EEE7FEE40E94662659
:101DD00011F00C94F10EEEE3F6E20E94C7230C948E
:101DE0009712E0E8FEE40E94662611F00C94FE0EC5
:101DF000E4E4F6E20E94C7230C949712E2E8FEE4C2
:101E00000E94662611F00C940B0FEAE4F6E20E94A1
:101E1000C7230C949712E4E8FEE40E94662611F0B2
:101E20000C94180FE6E7F7E20E94C7230C94971270
:101E3000E6E8FEE40E94662611F00C94250FE0E52A
:101E4000F6E20E94C7230C949712E8E8FEE40E9491
:101E5000662611F00C94320FE8E5F7E20E94C723E2
:101E60000C949712EAE8FEE40E94662611F00C94A6
:101E70003F0FE6E5F6E20E94C7230C949712ECE8C8
:101E8000FEE40E94662611F00C944C0FE2E8F7E2A3
:101E90000E94C7230C949712EEE8FEE40E94662687
:101EA00011F00C94590FEEE1F8E20E94C7230C9454
:101EB0009712E0E9FEE40E94662611F00C94660F8A
:101EC000ECE5F6E20E94C7230C949712E2E9FEE4E7
:101ED0000E94662611F00C94730FE2E6F6E20E946F
:101EE000C7230C949712E4E9FEE40E94662611F0E1
:101EF0000C94800FE8E8F7E20E94C7230C94971235
:101F0000E6E9FEE40E94662611F00C948D0FE4E2EF
:101F1000F8E20E94C7230C949712E8E9FEE40E94BD
:101F2000662611F00C949A0FEAE3F7E20E94C723A9
:101F30000C949712EAE9FEE40E94662611F00C94D4
:101F4000A70FE6EDF7E20E94C7230C949712ECE985
:101F5000FEE40E94662611F00C94B40FE0EAF7E26A
:101F60000E94C7230C949712EEE9FEE40E946626B5
:101F700011F00C94C10FE8E6F6E20E94C7230C941E
:101F80009712E0EAFEE40E94662611F00C94CE0F50
:101F9000EEE6F6E20E94C7230C949712E2EAFEE412
:101FA0000E94662611F00C94DB0FEAE5F8E20E942D
:101FB000C7230C949712E4EAFEE40E94662611F00F
:101FC0000C94E80FE8EBF7E20E94C7230C949712F9
:101FD000E6EAFEE40E94662611F00C94F50FE4E5B3
:101FE000F8E20E94C7230C949712E2E5FDE40E94F8
:101FF000662611F00C940210E4E7F6E20E94C72373
:102000000C949712E8EAFEE40E94662611F00C9404
:102010000F10EAE7F6E20E94C7230C949712E0E55E
:10202000FDE40E94662611F00C941C10ECE8F6E228
:102030000E94C7230C949712EAEAFEE40E946626E7
:1020400011F00C942910E2E9F6E20E94C7230C94E7
:102050009712ECEAFEE40E94662611F00C9436100A
:10206000E0E8F6E20E94C7230C949712EEEAFEE441
:102070000E94662611F00C944310E6E8F6E20E94F6
:10208000C7230C949712EEE4FDE40E94662611F03B
:102090000C945010E8E9F6E20E94C7230C949712C2
:1020A000E0EBFEE40E94662611F00C945D10EEE970
:1020B000F6E20E94C7230C949712ECE4FDE40E9420
:1020C000662611F00C946A10E4EAF6E20E94C72337
:1020D0000C949712E2EBFEE40E94662611F00C9439
:1020E0007710EAEAF6E20E94C7230C949712E4EB19
:1020F000FEE40E94662611F00C948410E0EDF7E2F5
:102100000E94C7230C949712E6EBFEE40E94662619
:1021100011F00C949110E0EBF6E20E94C7230C94AE
:102120009712E4E6FDE40E94662611F00C949E10DE
:10213000E6EBF6E20E94C7230C949712E8EBFEE46C
:102140000E94662611F00C94AB10ECEBF6E20E94B4
:10215000C7230C949712EAEBFEE40E94662611F066
:102160000C94B810E2ECF6E20E94C7230C9497128C
:10217000ECEBFEE40E94662611F00C94C510E8EC2E
:10218000F6E20E94C7230C949712EEEBFEE40E9445
:10219000662611F00C94D210EEECF6E20E94C723F2
:1021A0000C949712E0ECFEE40E94662611F00C9469
:1021B000DF10E4EDF6E20E94C7230C949712E2ECE4
:1021C000FEE40E94662611F00C94EC10EAEDF6E2B3
:1021D0000E94C7230C949712E4ECFEE40E9466264A
:1021E00011F00C94F910E0EEF6E20E94C7230C9473
:1021F0009712E6ECFEE40E94662611F00C9406119C
:10220000E6EEF6E20E94C7230C949712E8ECFEE497
:102210000E94662611F00C941311ECEEF6E20E9477
:10222000C7230C949712EAECFEE40E94662611F094
:102230000C942011E6E6F8E20E94C7230C94971252
:10224000ECECFEE40E94662611F00C942D11E2E7FE
:10225000F8E20E94C7230C949712EEECFEE40E9471
:10226000662611F00C943A11ECE6F8E20E94C723BE
:102270000C949712E0EDFEE40E94662611F00C9497
:102280004711E8E7F8E20E94C7230C949712E2EDA9
:10229000FEE40E94662611F00C945411EEEAF8E276
:1022A0000E94C7230C949712E4EDFEE40E94662678
:1022B00011F00C946111EEE7F8E20E94C7230C9430
:1022C0009712E6EDFEE40E94662611F00C946E1162
:1022D000E0ECF8E20E94C7230C949712E8EDFEE4CC
:1022E0000E94662611F00C947B11E4EEF8E20E9445
:1022F000C7230C949712EAEDFEE40E94662611F0C3
:102300000C948811EAEEF8E20E94C7230C9497120D
:10231000ECEDFEE40E94662611F00C949511E8EABB
:10232000F8E20E94C7230C949712EEEDFEE40E949F
:10233000662611F00C94A211ECEFF8E20E94C7237C
:102340000C949712E0EEFEE40E94662611F00C94C5
:10235000AF11E8E0F9E20E94C7230C949712E2EE75
:10236000FEE40E94662611F00C94BC11E8EDF8E240
:102370000E94C7230C949712E4EEFEE40E946626A6
:1023800011F00C94C911E4EBF8E20E94C7230C94FD
:102390009712E6EEFEE40E94662611F00C94D61128
:1023A000E6ECF8E20E94C7230C949712E8EEFEE4F4
:1023B0000E94662611F00C94E311E0E9F8E20E9415
:1023C000C7230C949712EAEEFEE40E94662611F0F1
:1023D0000C94F011E2EDF8E20E94C7230C949712DE
:1023E000ECEEFEE40E94662611F00C94FD11E0EF85
:1023F000F8E20E94C7230C949712EEEEFEE40E94CE
:10240000662611F00C940A12E4E8F8E20E94C72351
:102410000C949712E0EFFEE40E94662611F00C94F3
:102420001712EEEDF8E20E94C7230C949712E2EF28
:10243000FEE40E94662611F00C942412E2E0F9E218
:102440000E94C7230C949712E4EFFEE40E946626D4
:1024500011F00C943112E6E9F8E20E94C7230C94C3
:102460009712E6EFFEE40E94662611F00C943E12ED
:10247000EAEBF8E20E94C7230C949712E9EFF2E02E
:102480000E94682611F00C944B12ECECF8E20E94CA
:10249000C7230C949712E8EFFEE40E94662611F021
:1024A0000C945812E6EFF8E20E94C7230C9497129E
:1024B000EAEFFEE40E94662611F00C946512EAE849
:1024C000F8E20E94C7230C949712ECEFFEE40E94FE
:1024D000662611F00C947212E2EAF8E20E94C72319
:1024E0000C949712EEEFFEE40E94662611F00C9415
:1024F0007F12EEE0F9E20E94C7230C949712E0E00D
:10250000FFE40E94662611F00C948C12E4E1F9E2DB
:102510000E94C7230C949712E2E0FFE40E94662613
:1025200011F00C949712ECE9F8E20E94C72381E0C5
:10253000AA81BB818C93AA81BB810C91053018F0D4
:1025400011F00C94C5120E94CA23A881B9810E947F
:102550007A240C920E94C7235A924A92AA81BB8184
:102560008C91A42DB52D8C9381E00E94D1230E94E3
:10257000A709229681E00E94CD23AA81BB818C917C
:102580008F5F8C9310F40C949B1280E0A881B9812A
:102590008C935A924A92AA81BB818C91A42DB52D1D
:1025A0008C9381E00E94D1230E94A709229681E0AA
:1025B0000E94CD23AC81BD818C918F5F8C9310F4F0
:1025C0000C947B0ADE9A86E0481A8827580A2A96D5
:1025D00008957F49494931007C4A4A4931007F4981
:1025E000494936007C54542800007F010101030052
:1025F0007C0404040C00E0514F41FF00E0544C44C3
:10260000FC007C5554554400385554551800770843
:102610007F0877006C107C106C00414949493600F6
:102620004454545428007F1008047F007C20100874
:102630007C007F7F7F7F7F007842241278007C10AF
:102640002844000020413F017F0020443C047C00DE
:102650007C0810087C007C1010107C007F010101B8
:102660007F007C0404047C0004047C0404004728EC
:10267000100807007F7F7F7F7F000C1010107C0008
:102680000C127F120C0018247E2418007F7F7F7F9D
:1026900041007C404040FC007F7F7F4141007C4006
:1026A00078407C007F7F414141007C407840FC00C5
:1026B0007C50502000007F41414141004141414157
:1026C0004100414141417F007C5020007C0022417B
:1026D00049493E002844545438007F083E413E009A
:1026E0007C1038443800462919097F0008543414F6
:1026F0007C003E5149453E0000427F40000042615F
:10270000514946002241494936001814127F1000F1
:102710002745454539003E494949320061110905BF
:102720000300364949493600264949493E007E0999
:1027300009097E007F49494936003E414141220056
:102740007F4141413E007F49494941007F090909D4
:1027500001003E4149493A007F0808087F000041D6
:102760007F410000204141413F007F081422410089
:102770007F40404040007F0204027F007F04081039
:102780007F003E4141413E007F09090906003E416C
:1027900051617E007F0919294600064949493000E8
:1027A00001017F0101003F4040403F001F204020C9
:1027B0001F007F2010207F006314081463000304AF
:1027C0007804030061514945430020545454780073
:1027D0007F4844443800384444442800384444483E
:1027E0007F0038545454180000047E0500000C5239
:1027F000524A3C007F080404780000447D400000F9
:102800000040443D00007F201028440000417F40EC
:1028100000007C0418047C007C0804047800384420
:10282000444438007C1424241800182424147C0008
:102830007C0404080000085454542000043F444021
:1028400000003C4040407C001C2040201C003C40DC
:1028500030403C004428102844000C5050483C00B4
:102860004464544C4400000000000000006060001C
:1028700000000808080808000036360000000006BE
:1028800009090600007F414100000041417F00002E
:10289000552A552A550007097F0907004040404046
:1028A000400000563600000040400070700040407C
:1028B0000000000014141414140002015109060051
:1028C0007C7C0000000000005F00000000070007A3
:1028D0000000147F147F1400221408142200231314
:1028E000086462007C7C007F7F000005030000001C
:1028F000001C224100000041221C000014083E0878
:10290000140008083E0808000000503000002010A5
:10291000080402000204081020000000000000006B
:1029200000000000000000000080E0F8F8F8F0C0AF
:10293000000008081838F8F8F8F8F808080000004F
:102940000000000808F8F878180808000808D8F807
:10295000F8F8F8780808080818F8F8F0F0E000002F
:1029600000008888888888888888F800000000002F
:1029700000000000000000000000C0F03E0F010356
:102980000F3FFFFFFEF8E000000001071FFFFFFF01
:10299000FCF080000000C0F81F07010000000000EC
:1029A00080F8FFFFFF7F2760E0E0F0F8DC1F0F0FEB
:1029B0000701000000007844444444785048440033
:1029C00000000000000000008080C0E0F8FEC78129
:1029D0008101010101018187FFFFFFFFFCE0C08051
:1029E0008000031F7FFFFFFE7C0F030000000080BC
:1029F0008080C0F8FFFFFFFFCF80800001071F7FAE
:102A0000FFFFFCF0C080800000007C04080810205C
:102A100020407D00000000000000000000000000D9
:102A200000000808F8F8F8080000000000000000A6
:102A3000000000000000000000000000001818184E
:102A40000000000000000000000000000000000086
:102A500000000000000000000000000000003E2216
:102A60002222222222223E0000000000000000005C
:102A7000F8FCFE070181F1FFFF1F000078FCFE93C8
:102A800011190F8F46808E9E1F39F9F3E30301E180
:102A9000FFFF1F000000F8FCFE070301E1FEFF1F1F
:102AA000010181FFFF7F0602F1FFFF1E0000000011
:102AB00000009F909090909090909F0000000000E8
:102AC00000000000000101010100000101010100FE
:102AD00000000101010101000000010101010100EC
:102AE000000000000101010100000C1D1911191F57
:102AF0000F070100000001010100000000010101B9
:102B000001000000000010101010101010101F0025
:102B10000000A881B98188278C930E94E923A1E055
:102B2000B1E08C9300910101003011F00C949A15E2
:102B30000C94C4150D3011F00C94A0150C94C41510
:102B40000A3011F00C94AF15A881B9818C918030B6
:102B500011F40C94AD150C94C6150C94C415009189
:102B600001010F3118F011F00C94B8150C94C41534
:102B7000A1E0B1E08C91A881B9818F930E94DC2300
:102B80008F918D9388278C930C948D15089584E6EE
:102B900090E00E945F240E94E923A1E0B1E08C93C1
:102BA00000910101003011F00C94CB1508950E94A2
:102BB000E323A2E0B1E08C9300910201013011F017
:102BC0000C944417A2E3B2E0BA93AA930E94891529
:102BD0002296E2E3F2E004E0A3E0B1E00E942D26B9
:102BE000A3E0B1E0E4E0FFE40E94662611F00C945B
:102BF0003E17A2E3B2E00E946026EA2FFB2F339734
:102C0000F0400FEFA3E1B1E00E942D26E3E1F1E0F7
:102C100001E0A6E1B1E00E942D26A6E1B1E0E0EEE0
:102C2000FEE40E94662611F00C942316A2E3B2E0A3
:102C30000E946026EA2FFB2F3297F0400FEFA3E1AE
:102C4000B1E00E942D26E1E0F0E00E942824AFE9E7
:102C5000B0E088278C93EAE0FFE40E941A24A3E105
:102C6000B1E00E9414240E9421248AE090E00E9496
:102C70005F24A2E3B2E0BA93AA930E948915229638
:102C80008AE090E00E945F24A2E3B2E0BA93AA93A4
:102C90000E948915229686E1E2E3F2E00CE00A93B5
:102CA000AFE9B0E00E942626E2E3F2E0A8E1B1E05D
:102CB0000E9421268AE090E00E945F24A2E3B2E015
:102CC000BA93AA930E9489152296E2E3F2E0A8E162
:102CD000B1E00E942126E8E1F1E00EE0A8E1B1E0D8
:102CE0000E942D26DA9884E690E00E945F24DA9A0A
:102CF00082E390E00E945F24A7E7B2E08C918F5FAF
:102D00008C93009177020A3011F00C94721680E0D7
:102D1000809377025A924A9280E0A42DB52D8C932D
:102D200081E00E94D1235A924A9282E0A42DB52DCF
:102D30008C9381E00E94D1230E94B009249682E006
:102D40000E94CD235A924A92A42DB52DE4E1FFE4CE
:102D50000E9474248FE00E94D1230E94610A22966F
:102D60008FE00E94CD235A924A9280E0A42DB52D87
:102D70008C9381E00E94D1235A924A9282E0A42D42
:102D8000B52D8C9381E00E94D1230E94B009249636
:102D900082E00E94CD235A924A92EFE9F0E0A42DFE
:102DA000B52D0E9421268CE00E94D1230E94610A49
:102DB00022968CE00E94CD235A924A9280E0A42D64
:102DC000B52D8C9381E00E94D1235A924A9283E0E0
:102DD000A42DB52D8C9381E00E94D1230E94B009CF
:102DE000249682E00E94CD235A924A92A42DB52DBA
:102DF000E4E1FFE40E9474248FE00E94D1230E944A
:102E0000610A22968FE00E94CD235A924A9280E076
:102E1000A42DB52D8C9381E00E94D1235A924A9221
:102E200083E0A42DB52D8C9381E00E94D1230E94D4
:102E3000B009249682E00E94CD235A924A92E8E19A
:102E4000F1E0A42DB52D0E94212689E70E94D1230F
:102E50000E94610A229689E70E94CD23EEE9FDE4F3
:102E60000E941A2482E20E942424E8EAFDE40E94DF
:102E70001A2482E20E9424240E94212484E690E005
:102E80000E945F240E94C7150895A8E1B1E0E6ED15
:102E9000FDE40E94662611F00C948817969892988B
:102EA00080917A028F7780937A02ABE7B2E0E4E216
:102EB000FFE40E947424A8E1B1E088278C935A9221
:102EC0004A9280E0A42DB52D8C9381E00E94D123FD
:102ED0005A924A9283E0A42DB52D8C9381E00E94F2
:102EE000D1230E94B009249682E00E94CD235A92F9
:102EF0004A92A42DB52DE8E2FFE40E9474248FE0ED
:102F00000E94D1230E94610A22968FE00E94CD2365
:102F1000A8E1B1E0E8EDFDE40E94662611F00C9412
:102F2000CF17969AE8E2F0E00E942824929A8091C6
:102F30007A02806880937A02ABE7B2E0E8E3FFE4CC
:102F40000E947424A8E1B1E088278C935A924A9297
:102F500080E0A42DB52D8C9381E00E94D1235A925C
:102F60004A9283E0A42DB52D8C9381E00E94D12359
:102F70000E94B009249682E00E94CD235A924A9280
:102F8000A42DB52DECE3FFE40E9474248FE00E9491
:102F9000D1230E94610A22968FE00E94CD23A8E1EE
:102FA000B1E0EAEDFDE40E94662611F00C943418BD
:102FB0000E948F1EA8E1B1E088278C93AFE9B0E0B2
:102FC00088278C935A924A9280E0A42DB52D8C9339
:102FD00081E00E94D1235A924A9282E0A42DB52D1D
:102FE0008C9381E00E94D1230E94B009249682E054
:102FF0000E94CD235A924A92A42DB52DE4E1FFE41C
:103000000E9474248FE00E94D1230E94610A2296BC
:103010008FE00E94CD235A924A9280E0A42DB52DD4
:103020008C9381E00E94D1235A924A9283E0A42D8E
:10303000B52D8C9381E00E94D1230E94B009249683
:1030400082E00E94CD235A924A92A42DB52DE4E14C
:10305000FFE40E9474248FE00E94D1230E94610A41
:1030600022968FE00E94CD23A8E1B1E0ECEDFDE4D3
:103070000E94662611F00C9499180E944C1FA8E13A
:10308000B1E088278C93AFE9B0E088278C935A92FF
:103090004A9280E0A42DB52D8C9381E00E94D1232B
:1030A0005A924A9282E0A42DB52D8C9381E00E9421
:1030B000D1230E94B009249682E00E94CD235A9227
:1030C0004A92A42DB52DE4E1FFE40E9474248FE020
:1030D0000E94D1230E94610A22968FE00E94CD2394
:1030E0005A924A9280E0A42DB52D8C9381E00E94E3
:1030F000D1235A924A9283E0A42DB52D8C9381E07E
:103100000E94D1230E94B009249682E00E94CD2320
:103110005A924A92A42DB52DE4E1FFE40E94742452
:103120008FE00E94D1230E94610A22968FE00E94C4
:10313000CD23A8E1B1E0EEEDFDE40E94662611F09A
:103140000C94B6180E94D419E6E8F2E0A1E9B1E0C7
:103150000E942126E0E9F2E0A1E9B1E00E94DC232F
:103160000E9421260E9492190E94C715A8E1B1E091
:10317000E0EEFDE40E94662611F00C94C8188091E0
:103180007A028F7B80937A02A8E1B1E088278C9342
:10319000A8E1B1E0E2EEFDE40E94662611F00C9495
:1031A000DA1880917A02806480937A02A8E1B1E013
:1031B00088278C93A8E1B1E0ECE4FFE40E94662646
:1031C00011F00C940C19EFE9F0E0ADEDB2E00E94C3
:1031D0002126E0E0F0E0ADEDB2E07BE70E943B2687
:1031E000A1E9B1E0E8E5FFE40E947424EDEDF2E02E
:1031F000A1E9B1E00E94DC230E942126A1E9B1E00F
:103200000E94DC23E2E6FFE40E9474240E949219EB
:10321000A8E1B1E088278C93A8E1B1E0E6EFFEE4F5
:103220000E94662611F00C949119A1E9B1E0E6E63E
:10323000FFE40E9474248AE0A1E9B1E08F930E9428
:10324000DC238F918D9388278C93A1E9B1E00E94B4
:10325000DC23EEE6FFE40E947424E6E8F2E0A1E954
:10326000B1E00E94DC230E942126E0E9F2E0A1E91E
:10327000B1E00E94DC230E9421268AE0A1E9B1E0AE
:103280008F930E94DC238F918D9388278C93A1E9E3
:10329000B1E00E94DC23E4E7FFE40E947424EBE742
:1032A000F2E0A1E9B1E00E94DC230E9421268AE03D
:1032B000A1E9B1E08F930E94DC238F918D93882741
:1032C0008C93A1E9B1E00E94DC23EAE7FFE40E94CD
:1032D0007424EFE7F2E0A1E9B1E00E94DC230E9450
:1032E00021268AE0A1E9B1E08F930E94DC238F912F
:1032F0008D9388278C93A1E9B1E00E94DC23E6E856
:10330000FFE40E947424E1E8F2E0A1E9B1E00E9448
:10331000DC230E9421260E949219A8E1B1E08827AF
:103320008C930895EEE9FFE40E941A2482E20E9441
:103330002424ADEDB2E00E94142482E20E942424F1
:103340000E94212488EC90E00E945F24A1E9B1E072
:103350000E9414248AE10E9424240E9421248AE1EC
:103360000E942424E1E0F0E00E9428248DE00E94E5
:1033700024240E942124DA9884E690E00E945F24AD
:10338000DA9A82E390E00E945F24A7E7B2E08C9192
:103390008F5F8C93009177020A3011F00C94BB1967
:1033A00080E080937702089583E0E0E30E94D524D3
:1033B000002762FA0EF401E041E0041711F00C94CA
:1033C000161A8FEF80938502A6E8B2E0E8EAFFE4E0
:1033D0000E9474245A924A9280E0A42DB52D8C93B9
:1033E00081E00E94D1235A924A9281E0A42DB52D0A
:1033F0008C9381E00E94D1230E94B009249682E040
:103400000E94CD235A924A92E6E8F2E0A42DB52D0F
:103410000E94212686E00E94D1230E94610A229602
:1034200086E00E94CD2308950C94C01A6CEC83E0D2
:10343000E0E3BB27A6E121E02A930E94082564E48B
:1034400083E0E0E3BB27A6E121E02A930E94082560
:103450008EEE92E00E945F2483E0E0E30E94D52498
:103460006CEC83E0E0E3BB27A6E121E02A930E9415
:1034700008256EEB83E0E0E3BB27A6E121E02A9379
:103480000E940825BB27A6E183E0E0E321E02A9320
:103490000E943225ACE8B2E05C93BB27A6E183E052
:1034A000E0E321E02A930E943225ADE8B2E05C938C
:1034B00000918D02083F18F011F00C94611A0C94E1
:1034C000771A0FEF40918C02041BACE8B2E00C932A
:1034D0000FEF40918D02041BADE8B2E00C93A6E81B
:1034E000B2E0ECECFEE40E9474240C947D1AA6E891
:1034F000B2E0E2EFFEE40E94742400918C0240E10D
:103500000E945026AEE8B2E00C9300918D0240E19B
:10351000049FAFE8B2E00C9200918E0240918F02BE
:10352000040FA5E8B2E00C93A6E8B2E0ECECFEE4F0
:103530000E94662611F00C94A41A00918E0241E0BC
:10354000040FA5E8B2E00C93A6E8B2E0E2EFFEE4D7
:103550000E94662681E009F080E08F930091850249
:10356000003081E009F080E09F918923882311F4E5
:103570000C94C01AA6E8B2E0EAECFEE40E947424BF
:10358000A0E9B2E0E5E8F2E00E94A525E0E9F2E07A
:10359000ACE7B7E00E942126ECE7F7E0A0E9B2E053
:1035A0001127222700E033270E9488245A924A924A
:1035B00080E0A42DB52D8C9381E00E94D1235A92F6
:1035C0004A9281E0A42DB52D8C9381E00E94D123F5
:1035D0000E94B009249682E00E94CD235A924A921A
:1035E000A42DB52DE4E1FFE40E9474248FE00E9435
:1035F000D1230E94610A22968FE00E94CD235A9225
:103600004A9280E0A42DB52D8C9381E00E94D123B5
:103610005A924A9281E0A42DB52D8C9381E00E94AC
:10362000D1230E94B009249682E00E94CD235A92B1
:103630004A92E6E8F2E0A42DB52D0E94212686E00C
:103640000E94D1230E94610A229686E00E94CD2327
:103650005A924A9281E0A42DB52D8C9381E00E946C
:10366000D1235A924A9281E0A42DB52D8C9381E00A
:103670000E94D1230E94B009249682E00E94CD23AB
:103680005A924A92E0E9F2E0A42DB52D0E9421263B
:1036900085E00E94D1230E94610A229685E00E9463
:1036A000CD235A924A9283E0A42DB52D8C9381E0CC
:1036B0000E94D1235A924A9281E0A42DB52D8C9379
:1036C00081E00E94D1230E94B009249682E00E94EA
:1036D000CD235A924A92A42DB52DEEEAFFE40E9422
:1036E000742483E00E94D1230E94610A229683E021
:1036F0000E94CD230895E2EBFFE40E941A240E9469
:10370000212484EF91E00E945F24A2E3B2E0BA9307
:10371000AA930E948915229684E690E00E945F2475
:10372000A2E3B2E0BA93AA930E9489152296E2E33B
:10373000F2E0AEE9B2E00E9421268CE0EEE9F2E090
:1037400009E00A93AEE9B2E00E9426265A924A9214
:1037500080E0A42DB52D8C9381E00E94D1235A9254
:103760004A9280E0A42DB52D8C9381E00E94D12354
:103770000E94B009249682E00E94CD235A924A9278
:10378000A42DB52DECEBFFE40E9474248CE00E9484
:10379000D1230E94610A22968CE00E94CD235A9286
:1037A0004A9280E0A42DB52D8C9381E00E94D12314
:1037B0005A924A9280E0A42DB52D8C9381E00E940C
:1037C000D1230E94B009249682E00E94CD235A9210
:1037D0004A92EEE9F2E0A42DB52D0E94212685E162
:1037E0000E94D1230E94610A229685E10E94CD2386
:1037F0000E94C71508955A924A928BE0A42DB52DC8
:103800008C9381E00E94D1235A924A9280E0A42DA9
:10381000B52D8C9381E00E94D1230E94B00924969B
:1038200082E00E94CD235A924A92A42DB52DE4EF56
:10383000FEE40E94742482E00E94D1230E94610A67
:10384000229682E00E94CD23E8ECFFE40E941A2435
:103850000E9421248CE291E00E945F24A2E3B2E066
:10386000BA93AA930E948915229684E690E00E945A
:103870005F24A2E3B2E0BA93AA930E94891522962C
:10388000E2E3F2E0A6E9B2E00E94212687E0E6E961
:10389000F2E002E00A93A6E9B2E00E942626A6E939
:1038A000B2E00E94EF25ADE9B2E00C935A924A9241
:1038B0008CE0A42DB52D8C9381E00E94D1235A92E7
:1038C0004A9280E0A42DB52D8C9381E00E94D123F3
:1038D0000E94B009249682E00E94CD235A924A9217
:1038E000A42DB52DE0EDFFE40E94742483E00E9436
:1038F000D1230E94610A229683E00E94CD23009189
:103900009D02003080E010F009F081E08F9300917B
:103910009D02043081E008F080E09F918923882394
:1039200011F40C94BE1C5A924A928CE0A42DB52D31
:103930008C9381E00E94D1235A924A9280E0A42D78
:10394000B52D8C9381E00E94D1230E94B00924966A
:1039500082E00E94CD235A924A92A42DB52DE4ED27
:10396000FFE40E94742483E00E94D1230E94610A34
:10397000229683E00E94CD230C94B71D00919D02F6
:10398000043080E010F009F081E08F9300919D02F7
:10399000093081E008F080E09F918923882311F4A9
:1039A0000C94FD1C5A924A928CE0A42DB52D8C9358
:1039B00081E00E94D1235A924A9280E0A42DB52D35
:1039C0008C9381E00E94D1230E94B009249682E06A
:1039D0000E94CD235A924A92A42DB52DE8EDFFE422
:1039E0000E94742483E00E94D1230E94610A2296DF
:1039F00083E00E94CD230C94B71D00919D020930F5
:103A000080E010F009F081E08F9300919D020F306B
:103A100081E008F080E09F918923882311F40C94C1
:103A20003C1D5A924A928CE0A42DB52D8C9381E0D6
:103A30000E94D1235A924A9280E0A42DB52D8C93F6
:103A400081E00E94D1230E94B009249682E00E9466
:103A5000CD235A924A92A42DB52DECEDFFE40E949D
:103A6000742483E00E94D1230E94610A229683E09D
:103A70000E94CD230C94B71D00919D020F3080E071
:103A800010F009F081E08F9300919D02003281E0F7
:103A900008F080E09F918923882311F40C947B1D0A
:103AA0005A924A928CE0A42DB52D8C9381E00E940D
:103AB000D1235A924A9280E0A42DB52D8C9381E0B7
:103AC0000E94D1230E94B009249682E00E94CD2357
:103AD0005A924A92A42DB52DE0EEFFE40E94742480
:103AE00083E00E94D1230E94610A229683E00E9413
:103AF000CD230C94B71D00919D02003081E009F0A8
:103B000080E08F9300919D02033681E009F080E010
:103B10009F91892B882311F40C94B71D5A924A92D5
:103B20008CE0A42DB52D8C9381E00E94D1235A9274
:103B30004A9280E0A42DB52D8C9381E00E94D12380
:103B40000E94B009249682E00E94CD235A924A92A4
:103B5000A42DB52DE2EEFEE40E94742482E00E94C2
:103B6000D1230E94610A229682E00E94CD230E9406
:103B7000C7150895E4EEFFE40E941A240E94212450
:103B800080E991E00E945F24A2E3B2E0BA93AA9395
:103B90000E948915229680E991E00E945F24A2E3A9
:103BA000B2E0BA93AA930E948915229689E0E2E3D3
:103BB000F2E008E00A93A3EBB2E00E9426265A92B4
:103BC0004A9280E0A42DB52D8C9381E00E94D123F0
:103BD0005A924A9285E0A42DB52D8C9381E00E94E3
:103BE000D1230E94B009249682E00E94CD235A92EC
:103BF0004A92A42DB52DE4E1FFE40E9474248FE0E5
:103C00000E94D1230E94610A22968FE00E94CD2358
:103C10005A924A9280E0A42DB52D8C9381E00E94A7
:103C2000D1235A924A9285E0A42DB52D8C9381E040
:103C30000E94D1230E94B009249682E00E94CD23E5
:103C40005A924A92E3EBF2E0A42DB52D0E94212670
:103C500085E10E94D1230E94610A229685E10E949B
:103C6000CD2382E1E2E3F2E005E00A93A8ECB2E0C2
:103C70000E9426265A924A9280E0A42DB52D8C935C
:103C800081E00E94D1235A924A9284E0A42DB52D5E
:103C90008C9381E00E94D1230E94B009249682E097
:103CA0000E94CD235A924A92A42DB52DE4E1FFE45F
:103CB0000E9474248FE00E94D1230E94610A229600
:103CC0008FE00E94CD235A924A9280E0A42DB52D18
:103CD0008C9381E00E94D1235A924A9284E0A42DD1
:103CE000B52D8C9381E00E94D1230E94B0092496C7
:103CF00082E00E94CD235A924A92E8ECF2E0A42D91
:103D0000B52D0E94212685E10E94D1230E94610ADF
:103D1000229685E10E94CD230E94C7150895EEEEFC
:103D2000FFE40E941A24ADEDB2E00E941424ECEFEF
:103D3000FEE40E941A240E94212484E690E00E945E
:103D40005F245A924A9280E0A42DB52D8C9381E095
:103D50000E94D1235A924A9282E0A42DB52D8C93D1
:103D600081E00E94D1230E94B009249682E00E9443
:103D7000CD235A924A92A42DB52DE4E1FFE40E948E
:103D800074248FE00E94D1230E94610A22968FE062
:103D90000E94CD235A924A9280E0A42DB52D8C9397
:103DA00081E00E94D1235A924A9282E0A42DB52D3F
:103DB0008C9381E00E94D1230E94B009249682E076
:103DC0000E94CD235A924A92A42DB52DE2EFFFE432
:103DD0000E9474248AE00E94D1230E94610A2296E4
:103DE0008AE00E94CD235A924A9280E0A42DB52DFC
:103DF0008C9381E00E94D1235A924A9283E0A42DB1
:103E0000B52D8C9381E00E94D1230E94B0092496A5
:103E100082E00E94CD235A924A92A42DB52DE4E16E
:103E2000FFE40E9474248FE00E94D1230E94610A63
:103E300022968FE00E94CD235A924A9280E0A42DD0
:103E4000B52D8C9381E00E94D1235A924A9283E04F
:103E5000A42DB52D8C9381E00E94D1230E94B0093E
:103E6000249682E00E94CD235A924A92EDEDF2E030
:103E7000A42DB52D0E9421268DE00E94D1230E9401
:103E8000610A22968DE00E94CD23E4E1F0E00E94D9
:103E900028240E94C71508955A924A9280E0A42DC2
:103EA000B52D8C9381E00E94D1235A924A9282E0F0
:103EB000A42DB52D8C9381E00E94D1230E94B009DE
:103EC000249682E00E94CD235A924A92A42DB52DC9
:103ED000E4E1FFE40E9474248FE00E94D1230E9459
:103EE000610A22968FE00E94CD235A924A9280E086
:103EF000A42DB52D8C9381E00E94D1235A924A9231
:103F000082E0A42DB52D8C9381E00E94D1230E94E4
:103F1000B009249682E00E94CD235A924A92A42DA1
:103F2000B52DECEFFFE40E9474248FE00E94D123B2
:103F30000E94610A22968FE00E94CD235A924A92F3
:103F400080E0A42DB52D8C9381E00E94D1235A925C
:103F50004A9283E0A42DB52D8C9381E00E94D12359
:103F60000E94B009249682E00E94CD235A924A9280
:103F7000A42DB52DE4E1FFE40E9474248FE00E949B
:103F8000D1230E94610A22968FE00E94CD23ECE0AB
:103F9000F0E50E941A240E942124E1E0F0E00E9452
:103FA0002824A2E3B2E0BA93AA930E94891522962C
:103FB000A2E3B2E0BA93AA930E9489152296A2E3E3
:103FC000B2E0BA93AA930E9489152296E2E3F2E046
:103FD000A1E9B1E00E9421260E9492190E94C71512
:103FE00008955A924A9280E0A42DB52D8C9381E0D9
:103FF0000E94D1235A924A9283E0A42DB52D8C932E
:1040000081E00E94D1230E94B009249682E00E94A0
:10401000CD235A924A92A42DB52DE4E1FFE40E94EB
:1040200074248FE00E94D1230E94610A22968FE0BF
:104030000E94CD230027AAE7B2E08C9187FB0EF403
:1040400001E040E0041711F00C9457205A924A9274
:1040500080E0A42DB52D8C9381E00E94D1235A924B
:104060004A9283E0A42DB52D8C9381E00E94D12348
:104070000E94B009249682E00E94CD235A924A926F
:10408000A42DB52DE8E2FFE40E9474248FE00E9485
:10409000D1230E94610A22968FE00E94CD23ABE7D4
:1040A000B2E0E4E2FFE40E9474240C9486205A9269
:1040B0004A9280E0A42DB52D8C9381E00E94D123FB
:1040C0005A924A9283E0A42DB52D8C9381E00E94F0
:1040D000D1230E94B009249682E00E94CD235A92F7
:1040E0004A92A42DB52DECE3FFE40E9474248FE0E6
:1040F0000E94D1230E94610A22968FE00E94CD2364
:10410000ABE7B2E0E8E3FFE40E9474240027A0E3F9
:10411000B0E08C9184FB0EF401E040E0041711F054
:104120000C94E6205A924A9280E0A42DB52D8C93EF
:1041300081E00E94D1235A924A9282E0A42DB52DAB
:104140008C9381E00E94D1230E94B009249682E0E2
:104150000E94CD235A924A92A42DB52DE4E1FFE4AA
:104160000E9474248FE00E94D1230E94610A22964B
:104170008FE00E94CD235A924A9280E0A42DB52D63
:104180008C9381E00E94D1235A924A9282E0A42D1E
:10419000B52D8C9381E00E94D1230E94B009249612
:1041A00082E00E94CD235A924A92A42DB52DE6E1D9
:1041B000F0E50E9474248FE00E94D1230E94610ADE
:1041C00022968FE00E94CD230C944C215A924A9261
:1041D00080E0A42DB52D8C9381E00E94D1235A92CA
:1041E0004A9282E0A42DB52D8C9381E00E94D123C8
:1041F0000E94B009249682E00E94CD235A924A92EE
:10420000A42DB52DE4E1FFE40E9474248FE00E9408
:10421000D1230E94610A22968FE00E94CD235A92F8
:104220004A9280E0A42DB52D8C9381E00E94D12389
:104230005A924A9282E0A42DB52D8C9381E00E947F
:10424000D1230E94B009249682E00E94CD235A9285
:104250004A92A42DB52DE6E2F0E50E9474248CE08C
:104260000E94D1230E94610A22968CE00E94CD23F5
:10427000E2E0F0E00E9428240027A0E3B0E08C9167
:1042800084FB0EF401E041E0041711F00C944C2182
:104290000C947F000C944C210E94C7158AE090E09A
:1042A0000E945F2408950027A0E3B0E08C9187FB73
:1042B0000EF401E041E0041711F00C94FF215A9232
:1042C0004A9286E0A42DB52D8C9381E00E94D123E3
:1042D0005A924A9281E0A42DB52D8C9381E00E94E0
:1042E000D1230E94B009249682E00E94CD235A92E5
:1042F0004A92A42DB52DE2E3F0E50E94742489E0F2
:104300000E94D1230E94610A229689E00E94CD2357
:10431000AFE7B2E0E8EDFDE40E947424E1E0F0E0F4
:104320000E9428240027AAE7B2E08C9186FB0EF4B5
:1043300001E040E0041711F00C94FD21A1E9B1E087
:10434000ECE3F0E50E9474245A924A9280E0A42D96
:10435000B52D8C9381E00E94D1235A924A9281E03C
:10436000A42DB52D8C9381E00E94D1230E94B00929
:10437000249682E00E94CD235A924A92A42DB52D14
:10438000E4E1FFE40E9474248FE00E94D1230E94A4
:10439000610A22968FE00E94CD235A924A9280E0D1
:1043A000A42DB52D8C9381E00E94D1235A924A927C
:1043B00081E0A42DB52D8C9381E00E94D1230E9431
:1043C000B009249682E00E94CD235A924A92A42DED
:1043D000B52DE4E4F0E50E9474248FE00E94D1231F
:1043E0000E94610A22968FE00E94CD230E949219BA
:1043F00080917A02806480937A020C942E225A92E1
:104400004A9286E0A42DB52D8C9381E00E94D123A1
:104410005A924A9281E0A42DB52D8C9381E00E949E
:10442000D1230E94B009249682E00E94CD235A92A3
:104430004A92A42DB52DE4E5F0E50E94742489E0AC
:104440000E94D1230E94610A229689E00E94CD2316
:10445000AFE7B2E0E6EDFDE40E9474240027AAE78E
:10446000B2E08C9186FB0EF401E040E0041711F0FD
:104470000C946B225A924A928DE0A42DB52D8C9308
:1044800081E00E94D1235A924A9281E0A42DB52D59
:104490008C9381E00E94D1230E94B009249682E08F
:1044A0000E94CD235A924A92A42DB52DEAECFEE447
:1044B0000E94742482E00E94D1230E94610A229605
:1044C00082E00E94CD23A1E8B2E0EEE5F0E50E9493
:1044D00074240C949A225A924A928DE0A42DB52D00
:1044E0008C9381E00E94D1235A924A9281E0A42DBC
:1044F000B52D8C9381E00E94D1230E94B0092496AF
:1045000082E00E94CD235A924A92A42DB52DE6EE68
:10451000FEE40E94742482E00E94D1230E94610A7A
:10452000229682E00E94CD23A1E8B2E0E2E6F0E527
:104530000E9474240E94C7158AE090E00E945F24C4
:104540000895E6E6F0E50E941A240E9421248AE0FC
:1045500090E00E945F24A2E3B2E0BA93AA930E9483
:10456000891522968AE090E00E945F24A2E3B2E0DF
:10457000BA93AA930E948915229686E1E2E3F2E0BB
:104580000CE00A93AFE9B0E00E942626E2E3F2E0F5
:10459000A8E1B1E00E942126E8E1F1E004E0A8E111
:1045A000B1E00E942D26A8E1B1E0E0E7F0E50E942D
:1045B000662611F00C94C0238AE090E00E945F24EC
:1045C000A2E3B2E0BA93AA930E9489152296E2E38D
:1045D000F2E0A8E1B1E00E942126E8E1F1E00EE07E
:1045E000A8E1B1E00E942D26DA9884E690E00E94CE
:1045F0005F24DA9A82E390E00E945F24A7E7B2E0AA
:104600008C918F5F8C93009177020A3011F00C949B
:10461000F42280E0809377025A924A9280E0A42D9F
:10462000B52D8C9381E00E94D1235A924A9282E068
:10463000A42DB52D8C9381E00E94D1230E94B00956
:10464000249682E00E94CD235A924A92A42DB52D41
:10465000E4E1FFE40E9474248FE00E94D1230E94D1
:10466000610A22968FE00E94CD235A924A9280E0FE
:10467000A42DB52D8C9381E00E94D1235A924A92A9
:1046800082E0A42DB52D8C9381E00E94D1230E945D
:10469000B009249682E00E94CD235A924A92EFE913
:1046A000F0E0A42DB52D0E9421268CE00E94D1239C
:1046B0000E94610A22968CE00E94CD235A924A926F
:1046C00080E0A42DB52D8C9381E00E94D1235A92D5
:1046D0004A9283E0A42DB52D8C9381E00E94D123D2
:1046E0000E94B009249682E00E94CD235A924A92F9
:1046F000A42DB52DE4E1FFE40E9474248FE00E9414
:10470000D1230E94610A22968FE00E94CD235A9203
:104710004A9280E0A42DB52D8C9381E00E94D12394
:104720005A924A9283E0A42DB52D8C9381E00E9489
:10473000D1230E94B009249682E00E94CD235A9290
:104740004A92E8E1F1E0A42DB52D0E94212689E7E7
:104750000E94D1230E94610A229689E70E94CD23FC
:10476000EEE9FDE40E941A2482E20E942424E8EA91
:10477000FDE40E941A2482E20E9424240E94212443
:1047800084E690E00E945F240E94C71508958E2E53
:104790009F2E0895E82DF92D0895481A8827580A64
:1047A0000895480E8827581E0895ED91FC91EF5FFB
:1047B000FF4FFC93EE9308958F938D918823E9F733
:1047C00011978F91089580919E00882309F081E0D0
:1047D000089580919E00882309F408950F929F9375
:1047E000AF93BF937F9380919E008823E1F3F89469
:1047F00080919E008A9580939E0090919C00A0E6F7
:10480000B0E0A90F0024B01D8C9193959C3309F45E
:10481000992790939C0078947F91BF91AF919F913D
:104820000F900895ACE7B7E08D91882311F00CD07C
:10483000FBCF08950E947A24802D11F005D0FACF85
:1048400008958DE001D08AE05D9BFECF8CB908957C
:1048500088EE93E034D03197D9F708953197F1F786
:1048600008950E9441248D910E9445249A95D9F77C
:104870000E9444240895DB98D39ADC98D49AD19866
:104880000895DB98DC980895089508E0880F10F4E7
:10489000DC9A02C0DC980000DB9A0058005EF0F35E
:1048A000DB980058005EF0F3C99983950A9571F77B
:1048B0000895689462F80895E89462F80895EF9373
:1048C000FF93EE27E82BE92B31F0E0EAFFE0319788
:1048D000F1F70197D1F7FF91EF9108955A924A921B
:1048E000480E8827581E08950E947A240D920020B1
:1048F000D9F70895C89531960020089591E088234E
:1049000021F08894991F8A95E9F7892F9095089549
:104910002E2E3F2E992781918D3209F09395882371
:10492000D1F79A95E22DF32D112361F0091718F0B4
:1049300011F0101B01C0191B28F021F080E28D93AB
:104940001A95E9F780818D3219F48D93319604C060
:10495000222311F08BE28D93091738F031F0091BF7
:1049600021F080E38D930A95E9F781918D93882357
:10497000E1F7332351F0EA2FFB2F319633958E91D7
:1049800082933A95E1F78EE28C9308950181082B8A
:104990000183128119231283EF93FF93E4E0F0E087
:1049A0000E942E24FF91EF9108950E945924FF2721
:1049B0000E947E24EBDFEF93FF93ECE7F7E00E9489
:1049C0002E24FF91EF91182B128309230183EF937B
:1049D000FF93E4E6F1E00E942E24FF91EF91108115
:1049E000182369F4EF93FF93ECE7F7E00E942E247D
:1049F000FF91EF911081182311F00E945C24EF9336
:104A0000FF93ECE7F7E00E942E24FF91EF910895C9
:104A10000E947E24FF2729915D9148E0B7DFEF9344
:104A2000FF93E4E0F0E00E942E24FF91EF91579570
:104A300010F4182B1283EF93FF93ECEEF0E00E943A
:104A40002E24FF91EF91182B1283EF93FF93E4E054
:104A5000F0E00E942E24FF91EF914A95F9F62A95F5
:104A6000D9F608950E947E24FF27299148E0552712
:104A70008DDF09230183EF93FF93E4E1F0E00E94CF
:104A80002E24FF91EF9188941081182309F0089447
:104A90005795EF93FF93E0EBF0E00E942E24FF91F7
:104AA000EF914A9529F75D932A9501F708957F9331
:104AB0000F93AF93BF938F939F938FB78F938091F3
:104AC0009E000CE3081B21F49CB10E94592412C0E3
:104AD00000919D00A0E6B0E077279CB1A00FB71F22
:104AE0009C93839580939E0003950C3309F40027D3
:104AF00000939D008F918FBF9F918F91BF91AF9138
:104B00000F917F911895040F151F261F371F0895C9
:104B1000000F111F221F331F089500951095209537
:104B200030950F5F1F4F2F4F3F4F08950191108118
:104B30000EC001911191219130810BC00191108122
:104B400017FF05C03FEF2FEF04C000811127222778
:104B5000332737FF03C0E1DF8DE28D93CF93DF93DF
:104B6000CF92DF92EF92AA24BB24CC24DD24EE2442
:104B700040E2CAE0DD2755E093E38881890F87FD95
:104B80009F7083FD907F891B89935A95A9F7C0DF99
:104B9000AA1CBB1CCC1CDD1CEE1C4A9551F7E894EA
:104BA000EFE0FF2782910ED0EB30E0F71EF0689423
:104BB0008A2D0CD088278D93EF90DF90CF90DF91D6
:104BC000CF910895982F829501D0892F8F70805DA5
:104BD00026F0803309F4089568948D930895002792
:104BE0001127222733271DD08A3328F4803318F069
:104BF00005D015D0F9CF0EF490CF089580538F9340
:104C0000402F512F622F732F83DF82DF7CDF80DF05
:104C10008F919927080F191F291F391F08958D910A
:104C20000895E894FCDF8032E9F38B32D9F38930C0
:104C3000C9F38D3211F46894F2CF089588278D93CB
:104C4000089581918D938823E1F7089509919191B9
:104C5000992351F08A95D9F7319781918D930A95CF
:104C600019F08823D1F70895E9CFE199FECFEEBB83
:104C7000FFBB31960895F9DF8D917B3729F48DBB09
:104C8000E29AE19A8823B9F777270895EEDFE09A50
:104C90008DB38D93882319F09A95C1F79D9308954C
:104CA000FF93881BF9E0001FFA9511F4FF91089516
:104CB000881F841B18F4840F8894F5CF0894F3CFD1
:104CC0008FEF83959D919923E1F70895689401C032
:104CD000E894AF93BF938D9116F0919103C00E9419
:104CE0007A24902D891718F011F48823A1F7BF9129
:104CF000AF9108955265762E3132313033312E64C2
:104D0000000047534D2053494D39303044002D2D7C
:104D10002D2D2D2D2D2D2D2D2D2D2D2D00004156E0
:104D20005270726F6A6563742E727500C2EAEBFE90
:104D3000F7E5EDE8E520202020200000DAFAFAFA75
:104D4000FAFAFAFAFAFAFAFAFADB0000D900D8000D
:104D5000D600D700D0E5E3E8F1F2F0E0F6E8FF2076
:104D600020200000DA00CEF7E8F1F2EAE020E1F3DB
:104D7000F4E5F0E0000041540000C2E5F0E8F4E89A
:104D8000EAE0F6E8FF20415400004F4B0000D3E476
:104D9000E0EBE5EDE8E520534D53202000004154C1
:104DA0002B434D4744413D0044454C20414C4C0071
:104DB000C90053494D3930304420E3EEF2EEE22190
:104DC000000041542B434D47463D310041542B4395
:104DD0004C49503D31003000310032003300340086
:104DE00035003600370038003900410042004300EA
:104DF0004400450046004700480049004A004B0077
:104E00004C004D004E004F00500051005200530026
:104E10005400550056005700580059005A006100D0
:104E20006200630064006500660067006800690056
:104E30006A006B006C006D006E006F007000710006
:104E400072007300740075007600770078007900B6
:104E50007A00C000E000C100E100C200E200C3002F
:104E6000E300C400E400C500E500A800B800C600E7
:104E7000E600C700E700C800E800E900CA00EA0051
:104E8000CB00EB00CC00EC00CD00ED00CE00EE003E
:104E9000CF00EF00D000F000D100F100D200F2000E
:104EA000D300F300D500F500F700F600D400F400BD
:104EB000F800F900DC00FC00FA00DB00FB00DD007C
:104EC000FD00DE00FE00DF00FF0020002D002E00B0
:104ED0003A003E00B0004000260027003C002A00B7
:104EE0002C0024003D002100BD00230028005B00B1
:104EF00025002B005E003F005D0029003B002F00D5
:104F00005C005F002B434D54000041542B434D4740
:104F1000523D000020202020202020202020202082
:104F2000202000004F6666004C6F6164204F4646AB
:104F300020202020202000004F4E00004C6F616494
:104F4000204F4E2020202020202000004669727330
:104F5000746E756D626572004E756D6265723A2091
:104F60000000204F4B0053494D3930304400546508
:104F70006D703A004C6F61643A005049522073657D
:104F80006E736F723A0053656E6420534D53206602
:104F9000726F6D2073656E736F72733A00004154C7
:104FA0002B434D47533D00006572726F7200B04352
:104FB000000041542B434F50533F0000202020203D
:104FC000202020202020200041542B43535100005A
:104FD000202000003E2000003C2000003C4000005B
:104FE0003C26000041542B43434C4B3F00004154AE
:104FF0004400C7E2EEEDE8EC20EDE000C7E0EFF0A2
:10500000EEF120E1E0EBE0EDF1E000004154442A54
:1050100031303023000053494D39303044204F4E59
:1050200020202020000053494D39303044204F4685
:105030004600C4E0F22E203120200000416C617255
:105040006D210000CEF2EFF0E0E2EAE020534D5394
:1050500020200000C4E0F22E2030202000005965FE
:1050600073004E6F000041542B434D47523D3100B9
:065070002B434D47000038
:00000001FF
